:10000000ABEF0EF000000000EEEF0DF0000000007E
:0C001000000000000000000080EF0EF077
:10001C000B820BAE18EF00F00368026801680068F1
:08002C000A360232FF0E120039
:0E003400026A016A006A086A036A000E12007E
:100042000B840BAE2CEF00F0010E036E026A016A04
:0A005200006A0A360232FF0E1200A7
:08005C000AAE029E000E120024
:100064000CB074EF00F00CA21AEF01F00E6A000E4F
:1000740002648BEF00F0F00E0214D8A456EF00F0E7
:10008400023A01380F0B02260138F00B016E0038DA
:100094000F0B01260038F00B006E08380F0B0026FA
:1000A4000838F00B086E0E84D89002BE6FEF00F093
:1000B40008360036013602360E2A02BE6FEF00F013
:1000C40008360036013602360E2A02BE6FEF00F003
:1000D40008360036013602360E2A0E50036410EF3D
:1000E40001F0035E0BBC08AE15EF01F0D880800E62
:1000F40008640030000E002201220222D8A015EF6D
:1001040001F0023201320032034A1AEF01F015EF16
:1001140001F001C002F000C001F008C000F0086A5C
:10012400000E0E860264C2EF00F0F00E0214D8A492
:10013400AAEF00F0023A01380F0B02260138F00B47
:10014400016E00380F0B01260038F00B006E0E8490
:10015400D89002BE6FEF00F00036013602360E2A48
:1001640002BE6FEF00F00036013602360E2A02BEE0
:100174006FEF00F00036013602360E2A6FEF00F002
:1001840001C002F000C001F0006A000E0E960E8855
:100194000264EFEF00F0F00E0214D8A4DAEF00F0DE
:1001A400023A01380F0B02260138F00B016E0E845F
:1001B400D89002BE6FEF00F0013602360E2A02BE5E
:1001C4006FEF00F0013602360E2A02BE6FEF00F028
:1001D400013602360E2A6FEF00F001C002F0016A08
:1001E400000E0E8602641FEF01F0F00E0214D8A474
:1001F400FEEF00F0023A0E84D89002BE6FEF00F0DA
:1002040002360E2A02BE6FEF00F002360E2A02BE3C
:100214006FEF00F002360E2A6FEF00F0010E0C6E45
:100224000EDF22EF01F0020E0C6E16DF22EF01F05A
:10023400040E0C6EF1DE22EF01F0080E0C6EF8DEF7
:020244001200A6
:1002460000000000000000000000000000000000A8
:0802560000000000000012008E
:10025E002DC3C9FFC7B002D00000FCD7C9CF00F034
:02026E0012007C
:100270008B90350E0D6E0D2EFED724C32DF3EFDFC0
:1002800025C32DF3ECDFDFDF24C32DF3E8DF26C326
:100290002DF3E5DFD8DF24C32DF3E1DF27C32DF3F2
:1002A000DEDFD1DF24C32DF3DADF28C32DF3D7DF60
:1002B000CADF24C32DF3D3DF29C32DF3D0DFC3DF7F
:1002C00024C32DF3CCDF2AC32DF3C9DFBCDF24C345
:1002D0002DF3C5DF2BC32DF3C2DFB5DF24C32DF310
:0E02E000BEDF2CC32DF3BBDFAEDF8B80120020
:1002EE00025006180E6E086A096A0B6A03500764FC
:1002FE006AEF02F006500A6E068E028E03500B6EE7
:10030E000750036E000E0B64BAEF01F00B50075E40
:10031E00D8B45BEF02F0070E076429EF02F0075E18
:10032E0000C008F001C000F002C001F0026A074EE2
:10033E005BEF02F00764FEEF01F0075E00C008F00D
:10034E0001C000F0016A074E5BEF02F00764DCEFBC
:10035E0001F0075E00C008F0006A074E5BEF02F086
:10036E000764C3EF01F00AC002F005C001F004C03B
:10037E0000F0086A84EF03F0030E0764CEEF01F07D
:10038E00075E08380F0B086E074E5BEF02F0D89031
:10039E000832074E5BEF02F0D8900832074E5BEF43
:1003AE0002F0D89008325BEF02F0030E0764EDEF17
:1003BE0001F0075E08380F0B086E0038F00B0826A8
:1003CE0000380F0B006E074E5BEF02F0D890003234
:1003DE000832074E5BEF02F0D89000320832074E1B
:1003EE005BEF02F0D890003208325BEF02F0030EA2
:1003FE00076415EF02F0075E08380F0B086E003821
:10040E00F00B082600380F0B006E0138F00B00269B
:10041E0001380F0B016E074E5BEF02F0D8900132E0
:10042E0000320832074E5BEF02F0D89001320032F4
:10043E000832074E5BEF02F0D890013200320832DC
:10044E005BEF02F0030E076446EF02F0075E08381A
:10045E000F0B086E0038F00B082600380F0B006EDD
:10046E000138F00B002601380F0B016E0238F00B2D
:10047E00012602380F0B026E074E5BEF02F0D8908A
:10048E000232013200320832074E5BEF02F0D89092
:10049E000232013200320832074E5BEF02F0D89082
:1004AE000232013200320832096A000E0EAE4FEFF0
:1004BE0003F0081E001E011E021E082A0022012241
:1004CE0002224FEF03F00750D8A470EF02F084EF32
:1004DE0003F0096A02C00AF0028E068E0750035C12
:1004EE00076ED8B442EF03F0070E076410EF03F067
:1004FE00075E0450096E0550046E0650056E066ABE
:10050E00074E42EF03F0070E0764E5EF02F0075EB9
:10051E000450096E0550046E056A074E42EF03F053
:10052E00070E0764C3EF02F0075E0450096E046AFB
:10053E00074E42EF03F0070E0764AAEF02F00AC05F
:10054E0002F084EF03F0030E0764B5EF02F0075ECE
:10055E0009380F0B096E074E42EF03F0D89009329F
:10056E00074E42EF03F0D8900932074E42EF03F0E8
:10057E00D890093242EF03F0030E0764D4EF02F075
:10058E00075E09380F0B096E0438F00B0926043884
:10059E000F0B046E074E42EF03F0D890043209326F
:1005AE00074E42EF03F0D89004320932074E42EF65
:1005BE0003F0D8900432093242EF03F0030E0764C1
:1005CE00FCEF02F0075E09380F0B096E0438F00BD2
:1005DE00092604380F0B046E0538F00B0426053877
:1005EE000F0B056E074E42EF03F0D8900532043222
:1005FE000932074E42EF03F0D89005320432093229
:10060E00074E42EF03F0D89005320432093242EF22
:10061E0003F0030E07642DEF03F0075E09380F0B8E
:10062E00096E0438F00B092604380F0B046E0538DA
:10063E00F00B042605380F0B056E0638F00B052659
:10064E0006380F0B066E074E42EF03F0D8900632B7
:10065E00053204320932074E42EF03F0D8900632CB
:10066E00053204320932074E42EF03F0D8900632BB
:10067E00053204320932086A000E0EAE4FEF03F057
:10068E00091E041E051E061E092A04220522062224
:10069E00095008260450002205500122065002225D
:1006AE000EBE66EF03F0D8A075EF03F002320132F2
:1006BE0000320832033E75EF03F07FEF03F0D8B03F
:1006CE007AEF03F0000E081E001E011E021E082AFD
:1006DE000022012202220A7E7AEF03F0010E0C6E36
:1006EE00BADC86EF03F0020E0C6EB5DC86EF03F07B
:1006FE00040E0C6E8CDC86EF03F0000E0C6E1200F6
:10070E000C6A0E6A0250D8A4A0EF03F001C002F0EA
:10071E0000C001F0006A0E860250D8A4A0EF03F0CC
:10072E0001C002F0016A0E960E880250D8B4B2EFE4
:10073E0003F00E50035ED8A4D8A0B7EF03F0D89004
:10074E0002BEBCEF03F0003601360236032EA7EFD1
:10075E0003F0B7EF03F0010E0C6E65DCBFEF03F094
:10076E00020E0C6E67DCBFEF03F0040E0C6E6FDC36
:02077E00120067
:100780000B800BAECCEF03F0026A0AAEFF0E026ED6
:0C079000016E006E0A360232FF0E1200ED
:08079C000B6A0B86FF0E120030
:0A07A400750E0D6E0D2EFED712002B
:1007AE0003011A6B080E1A5D0FE21A51010F246F26
:1007BE00256B266B276B286B296B2A6B2B6B2C6B8F
:0A07CE0050DD03011A2BEED71200D4
:1007D8000B6A0350D8B432EF04F002500A6E028E4E
:1007E8008E0E035E03AE36EF04F0036C080E035C56
:1007F800D8A011EF04F0036E013602C001F0026ABE
:10080800080E035CD8A011EF04F0036E0136016AEC
:100818000350D8A4D8901BEF04F00350D8B41BEFB2
:1008280004F0D89002320132032E15EF04F00BBC0D
:1008380001A028EF04F0D8A028EF04F0012AD8B4CA
:10084800022A02BE45EF04F00AAE4AEF04F0021E87
:10085800011E012AD8B4022A4AEF04F0026A016A8A
:100868004AEF04F00B800BAE4EEF04F0026A0AAEBA
:100878004EEF04F0FF0E026E016E0A3602324EEFA2
:1008880004F0010E0C6E78DF50EF04F0000E0C6ED1
:1008980050EF04F0FF0E0C6E0150006E0250016E16
:0208A80012003C
:1008AA00086A080E0C6E003408360450085ED8B088
:0E08BA0002D00826D89000360C2EF5D712007A
:0E08C800ACB202D00000FCD71AC3ADFF120084
:1008D600086A096A000E07620364F0EF04F002502A
:1008E60006180A6E075003267E0ED8A081EF04F084
:1008F600035ED8B0F5EF04F085EF04F0035ED8A0F0
:10090600FAEF04F0028E068E02C00EF001C00BF064
:1009160000C00DF000500402F4CF0CF001500502A7
:10092600F4CF00F0F3CF08F00402F3500C26F45095
:100936000822000E00220D500502F3500C26F4503A
:100946000822000E002202500402F3500826F4503A
:10095600002202500502016A000E0122F350002611
:10096600F45001220D500602F3500826F4500022DE
:10097600026A000E012202220B500602F3500026E4
:10098600F4500122000E02220E500602F3500126F8
:10099600F450022202BED8EF04F0083600360136C3
:1009A60002360306D8B4FAEF04F0EBEF04F0D88071
:1009B600800E08640030000E002201220222D8A018
:1009C600EBEF04F0023201320032034AF5EF04F095
:1009D6000AAE029E000EFDEF04F0010E1AEC00F0C6
:1009E600FDEF04F0020E0EEC00F0FDEF04F0040E35
:0609F60021EC00F01200EC
:1009FC000450000A12E10550000A0FE10650000AEB
:100A0C000CE10750000A09E1FF0E006EFF0E016EAB
:100A1C007F0E026EFF0E036EA7D0086A096A07509C
:100A2C00D8B4A9EF05F00350D8B4ADEF05F00250DF
:100A3C0006180A6E028E068E0E6A02C008F001C0FD
:100A4C000CF000C00DF004500D5E0550D8A0053C14
:100A5C000C5E0650D8A0063C085E086A0C6A0D6A4B
:100A6C00D8A040EF05F0D8900232013200320832A3
:100A7C00010E0E6E0750035ED8A04DEF05F07E0EF2
:100A8C000E240326D8B0B2EF05F053EF05F07E0E1E
:100A9C000E240326D8A0B7EF05F0180E0B6E0D36FA
:100AAC000C3608360036013602360E360450005E1F
:100ABC000550D8A0053C015E0650D8A0063C025E4D
:100ACC0006340E120EA06EEF05F00D8079EF05F0D6
:100ADC00045000260550D8B0053C01260650D8B06D
:100AEC00062802260D900B2E55EF05F09FEF05F012
:100AFC00D8900036013602360E360450005E055092
:100B0C00D8A0053C015E0650D8A0063C025E063417
:100B1C000E10010B0D26D8B00C2AD8B4082AD8A474
:100B2C009FEF05F008320C320D32032AD8B4B2EF25
:100B3C0005F00AAE089E0850026E0C50016E0D5066
:100B4C00006EBAEF05F0010E23DEBAEF05F0020ECF
:100B5C001AEC00F0BAEF05F0040E0EEC00F0BAEF50
:0A0B6C0005F0080E21EC00F0120065
:100B76001AC3E9FF1BC3EAFFEE5003011C1905E186
:100B86001AC300F01BC301F010D01AC300F01BC338
:100B960001F01A4B1B2B00C0E9FF01C0EAFFEECFA4
:0C0BA60000F00052E5E1006A016A120054
:100BB20003011A51390806E3300E1A5D03E3010EF0
:080BC200006E01D0006A120070
:100BCA000B6A0A6A096A00500402F4CF09F0F3CFEB
:100BDA0008F001500502F4CF0BF0F3CF0AF00050F1
:100BEA000502F3500926F4500A22E86A0B22015042
:100BFA000402F3500926F4500A22E86A0B2208C0BC
:100C0A0000F009C001F00AC002F00BC003F01200A4
:100C1A001EC300F003011E07005228E01AC3E9FFB1
:100C2A001BC3EAFFEE50000A0CE01AC3E9FF1BC31C
:100C3A00EAFF1CC3D9FF1DC3DAFFEE50DE1801E13B
:100C4A000FD01AC3E9FF1BC3EAFF1CC3D9FF1DC398
:100C5A00DAFFDE50EE5C006E016A000E015A08D01F
:100C6A0003011A4B1B2B1C4B1D2BD2D7006A016A9E
:020C7A00120066
:100C7C0000C008F00150006E016A026A036A0B6A38
:100C8C000C6A016A026A036A960E036E0A6A00AE67
:100C9C0056EF06F0081E001E082AD8B4002A0A8E49
:100CAC0000C001F008C000F0086A026A2ADD1200D8
:080CBC00067E77EC01F0120046
:100CC4001AC302F01BC303F002C000F003C001F01A
:100CD400024A032A00C0E9FF01C0EAFFEE5201E024
:100CE400F3D703011A51025C006E1B510358016EC5
:0A0CF400010E005E000E015A12000E
:100CFE000A6A0350D8A40A800750D8A40A820A5060
:100D0E00D8B4E2EF06F0030AD8B49BEF06F00AB0AF
:100D1E0096EF06F006AEE0EF06F0DEEF06F002AE5E
:100D2E00DEEF06F0E0EF06F00250800B0A6E029E38
:100D3E000650800B069E0A18D8B4ACEF06F00A5087
:100D4E00D8B4DEEF06F0E0EF06F00750035CD8B43F
:100D5E00B6EF06F0D8A0D2EF06F0D8EF06F00650A8
:100D6E00025CD8B4C0EF06F0D8A0D2EF06F0D8EFF0
:100D7E0006F00550015CD8B4CAEF06F0D8A0D2EF49
:100D8E0006F0D8EF06F00450005CD8B4E2EF06F09F
:100D9E00D8B0D8EF06F00A52D8B4E0EF06F0DEEF86
:100DAE0006F00A52D8B4DEEF06F0E0EF06F0D88077
:0E0DBE001200D8901200D880D88412001200C3
:100DCC00030E006E1AC321F3000E0301226F0050B4
:100DDC0005E0213721912237FF0FFAD7236B320E12
:100DEC001A25F66E290EF76E000EF722000EF86E1D
:100DFC00000EF822F6CFF6FFF7CFF7FFF8CFF8FF8B
:100E0C000900F5CF81F11F6B206B000E205D02E114
:100E1C00080E1F5DD8B002D1400E1D6F000E1E6F64
:100E2C00000E006E1E51005C02E11D51000821E213
:100E3C00810E1D25E16E010E1E21E26E010E1D5D5F
:100E4C00006E000E1E59016E810E0024E96E010E1B
:100E5C000120EA6EE9CFE9FFEACFEAFFE1CFE1FF3B
:100E6C00E2CFE2FFEECFE6FF010E1D5F000E1E5B30
:100E7C00D7D721511F25006E22512021016E320E31
:100E8C000024F66E290E0120F76E000EF86E000E8F
:100E9C00F822F6CFF6FFF7CFF7FFF8CFF8FF0900EF
:100EAC00F5CF81F1236B080E1D6F000E1E6F000E27
:100EBC00006E1E51005C02E11D510008D8B097D0A5
:100ECC001DC324F3810EE96E010EEA6E2351E9264F
:100EDC00D8B0EA2AE9CFE9FFEACFEAFFEECF25F353
:100EEC00080E2325006E016A000E0122810E0024DB
:100EFC00E96E010E0120EA6EE9CFE9FFEACFEAFFC5
:100F0C00EECF26F3100E2325006E016A000E01228F
:100F1C00810E0024E96E010E0120EA6EE9CFE9FF93
:100F2C00EACFEAFFEECF27F3180E2325006E016AF5
:100F3C00000E0122810E0024E96E010E0120EA6EE2
:100F4C00E9CFE9FFEACFEAFFEECF28F3200E232505
:100F5C00006E016A000E0122810E0024E96E010E62
:100F6C000120EA6EE9CFE9FFEACFEAFFEECF29F3E1
:100F7C00280E2325006E016A000E0122810E00242A
:100F8C00E96E010E0120EA6EE9CFE9FFEACFEAFF34
:100F9C00EECF2AF3300E2325006E016A000E0122DB
:100FAC00810E0024E96E010E0120EA6EE9CFE9FF03
:100FBC00EACFEAFFEECF2BF3380E2325006E016A41
:100FCC00000E0122810E0024E96E010E0120EA6E52
:100FDC00E9CFE9FFEACFEAFFEECF2CF338EC01F0D2
:100FEC000301232B010E1D5F000E1E5B60D71D6BD2
:100FFC001E6B1C511E5D02E11B511D5D0CE2150E9A
:10100C000C6EC60E0D6E0D2EFED70C2EFCD70000EE
:0E101C001D4B1E2BEED71F4B202BF7D61200BC
:10102A00086A096A100E0C6E013408360936045033
:10103A00085E0550D8A0053C095ED8B007D0045018
:10104A0008260550D8B0053C0926D8900036013646
:06105A000C2EEAD7120083
:10106000C280C19EC08EC08AC088C096C082C09413
:0C107000C090C196C194C192C1901200C2
:10107C000301056B03C3E9FF04C3EAFFEECF00F1E4
:10108C0001010051000A0EE000C11AF317DC030144
:10109C00052B05510325E96E000E0421EA6EEECFF7
:0610AC0000F1EED7120076
:1010B20005C304F006C305F003C302F004C303F042
:1010C20007C300F008C301F0010E0301075F000E21
:1010D200085B005001100FE004C0E9FF05C0EAFF01
:1010E20002C0E1FF03C0E2FFEECFE6FF024A032A9D
:1010F200044A052AE5D703C300F004C301F0120035
:101102000101006B050E005D0CE200510301052593
:10111200E16E000E0621E26E200EE66E0101002B4A
:10112200F1D7005103010525E16E000E0621E26EA2
:10113200E66A01010007005103010525076F000E51
:101142000621086F0A0E046E000E056E03C300F03E
:1011520004C301F069DF08C000F009C001F0300EDD
:10116200002607C3E1FF08C3E2FF00C0E6FF0A0E44
:10117200046E000E056E03C300F004C301F054DFD9
:1011820000C003F301C004F3000E011802E1000ED7
:0E119200001801E103D001010007CDD71200C3
:1011A000C80E0101616F080E626F1A0E636F030EA5
:1011B000646FFF0E656FFF0E666F000E676F000EA7
:1011C000686FFF0E596FFF0E5A6F000E5B6F000EB7
:1011D0005C6FFF0E5D6FFF0E5E6F000E5F6F000EA7
:1011E000606FAC8A900EAB6E948E949C9EAA03D0D6
:0811F000AECF00F0FBD71200A6
:1011F800130E806E0F01386B38813883170E926E8C
:10120800929A899A806A546BFF0E816E830E936E50
:10121800396B826A3A6BFF0E946E948E949C94900C
:101228008B80836A3B6BFF0E956E95909482959C9C
:06123800948E606A1200B2
:10123E000900F5CFE6FF0006FBE10106F9E1120019
:10124E0005C3F6FF06C3F7FF07C3F8FF0900F5CF86
:10125E0000F0005218E005C3F6FF06C3F7FF07C300
:10126E00F8FF0900F5CF00F003C3E1FF04C3E2FF6E
:10127E0000C0E6FF0301034B042B010E0527000EF1
:10128E0006230723DDD703C3E1FF04C3E2FFE66AAB
:02129E0012003C
:1012A00003C3F6FF04C3F7FF05C3F8FF0900F5CF3A
:1012B00000F0005212E003C3F6FF04C3F7FF05C3BA
:1012C000F8FF0900F5CF1AF364EC04F0010E0301F6
:0C12D0000327000E04230523E3D71200BF
:1012DC000D0E03011A6F64EC04F00A0E03011A6F71
:0612EC0064EC04F01200A6
:1012F200C26A00017F1D006E0050C1160F0EC0129F
:10130200C08E00C100F00036009000360090005000
:10131200C212C280D2EC03F0C282C2A201D0FDD7B7
:10132200C4CF01F0006A00C003F301C004F3C3504C
:101332000012000E011200C003F301C004F3C290B8
:10134200000E0014026E0150800B036E000E031893
:1013520002E1000E021803E00301036B046B03C3F6
:0813620000F004C301F01200C9
:10136A0003C304F004C305F004C0E9FF05C0EAFFA3
:10137A00EE5203E0044A052AF7D704C002F005C07A
:10138A0003F0044A052A05C300F006C301F003016D
:10139A00054B062B00C0E9FF01C0EAFF02C0E1FFCE
:1013AA0003C0E2FFEECFE6FF02C0E9FF03C0EAFF97
:1013BA00EE5201E0E2D703C300F004C301F01200C9
:1013CA00000E0301041902E1000E031935E003C3FC
:1013DA00E9FF04C3EAFFEE522FE005C31AF306C37E
:1013EA001BF36BDC00C01EF303C31AF304C31BF325
:1013FA0005C31CF306C31DF30BDC000E011802E142
:10140A00000E001805E103C300F004C301F016D072
:10141A00010E030103251A6F000E04211B6F05C379
:10142A00E9FF06C3EAFFEECF1CF3BBEC05F000C0F0
:0E143A0003F301C004F3C4D7006A016A120074
:1014480003C3E9FF04C3EAFFEE5000080EE203C33A
:10145800E9FF04C3EAFFEECF1AF305C31BF306C383
:0C1468001CF3B0DC034B042BEBD712008C
:1014740003010951000805E3070E0A6F000E0B6F04
:1014840012D00951160805E2170E0C6F000E0D6FED
:1014940006D00951010F0C6F0D6B000E0D230CC308
:1014A4000AF30DC30BF30AC314F30BC315F30E6B4A
:1014B4000F6B046A056A066A076A03C300F004C373
:1014C40001F005C302F006C303F017DC010ED8B027
:1014D400000E006E005209E007C3E1FF08C3E2FFFB
:1014E4002D0EE66E074B082B057F03C304F004C3DF
:1014F40005F005C306F006C307F0006A016A026A34
:10150400036A7FEC06F0010ED8B0000E006E0052A4
:1015140037E0000E046E000E056E000E066E7F0EA0
:10152400076E03C300F004C301F005C302F006C351
:1015340003F07FEC06F0010ED8B0000E006E0052EE
:101544001FE003C300F004C301F005C302F006C3A7
:1015540003F0000E046E000E056E200E066E820E61
:10156400076E6BEC04F000C003F301C004F302C087
:1015740005F303C006F3010E0E5F000E0F5BC9D71F
:10158400000E046E000E056E200E066E820E076EAF
:1015940003C300F004C301F005C302F006C303F063
:1015A4007FEC06F0000ED8B0010E006E00521EE073
:1015B400000E046E000E056E200E066E820E076E7F
:1015C40003C300F004C301F005C302F006C303F033
:1015D400FEEC04F000C003F301C004F302C005F301
:1015E40003C006F303010E4B0F2BCAD70E51142769
:1015F4000F511523010E106F000E116F000E166FA0
:10160400000E176F000E186F7F0E196F800E1119E0
:10161400006E800E1519005C02E11451105D1EE28B
:10162400000E046E000E056E200E066E820E076E0E
:1016340016C300F017C301F018C302F019C303F076
:10164400FEEC04F000C016F301C017F302C018F357
:1016540003C019F30301104B112BD8D7000E046EED
:10166400000E056E000E066E800E076E16C300F0A7
:1016740017C301F018C302F019C303F0FEEC04F021
:1016840003C304F004C305F005C306F006C307F062
:1016940077EC01F000C003F301C004F302C005F3CA
:1016A40003C006F3000E046E000E056E200E066ED7
:1016B400820E076E7FEC06F0000ED8B0010E006EAD
:1016C40000520BE0000E0301036F000E046F000EC6
:1016D400056F7F0E066F0E4B0F2B0301800E0F1943
:1016E400006E800E005C02E1000E0E5D38E207C35E
:1016F400E1FF08C3E2FF300EE66E074B082B07C379
:10170400E1FF08C3E2FF2E0EE66E074B082B800EA6
:101714001519006E800E005C02E1000E145D04E2F7
:1017240014510E5F15510F5BFF0E106FFF0E116FFA
:10173400800E0F19006E800E1119005C02E1105129
:101744000E5D0DE207C3E1FF08C3E2FF300EE66E53
:10175400074B082B010E105F000E115BE9D7106BCD
:10176400116B800E1119006E800E1519005C02E1D8
:101774001451105D63E203C300F004C301F005C318
:1017840002F006C303F0ECEC03F000C012F301C056
:1017940013F3300E002607C3E1FF08C3E2FF00C0C5
:1017A400E6FF074B082B11510F1902E10E511019D6
:1017B40008E107C3E1FF08C3E2FF2E0EE66E074B04
:1017C400082B12C300F013C301F03EEC06F000C076
:1017D40016F301C017F302C018F303C019F300C0D5
:1017E40004F001C005F002C006F003C007F003C313
:1017F40000F004C301F005C302F006C303F05EEC7D
:1018040006F000C003F301C004F302C005F303C0F3
:1018140006F3000E046E000E056E200E066E820E98
:10182400076E6BEC04F000C003F301C004F302C0C4
:1018340005F303C006F3104B112B93D707C3E1FF45
:0818440008C3E2FFE66A12008E
:10184C0001017F6B806B000E805D02E1800E7F5D7D
:10185C0016E2810E7F25E16E020E8021E26EE1CF51
:10186C00E1FFE2CFE2FFE66A010E7F25006E000E7B
:10187C008021016E00C07FF101C080F1E4D77F6B45
:10188C00806B0301016B026BAECFFFF00001FF6BAD
:0A189C000101016B026B9D8A12002E
:1018A60003C3E9FF04C3EAFFEECF05F3000E03010D
:1018B600066F000E066F000E061902E1200E0519CE
:1018C60007E0000E061902E1090E051901E003D032
:1018D600034B042BE5D7076B086B096B0A6B000EED
:1018E600061902E12D0E051905E1094B0A2B034BDA
:1018F600042B08D0000E061902E12B0E051902E191
:10190600034B042B03C3E9FF04C3EAFFEECF05F341
:10191600000E066F000E066F05C31AF3D9EC05F02C
:10192600005219E007C300F008C301F00A0E046E66
:10193600000E056EE5EC05F0300E055D026E000E3C
:101946000659036E02500024076F03500120086FEA
:10195600034B042BD7D709510A1108E00751000899
:10196600006E08C301F0000E015604D007C300F054
:0619760008C301F012009D
:10197C008B90090E0301246F256B266B276B286B4C
:10198C00296B2A6B2B6B2C6B38EC01F00A0E0301C4
:10199C00246F010E256F010E266F010E276F010EAD
:1019AC00286F010E296F010E2A6F010E2B6F010E8D
:1019BC002C6F38EC01F00B0E0301246F070E256F12
:1019CC00070E266F070E276F070E286F070E296F5D
:1019DC00070E2A6F070E2B6F070E2C6F38EC01F0D9
:1019EC000C0E0301246F010E256F010E266F010EE4
:1019FC00276F010E286F010E296F010E2A6F010E41
:101A0C002B6F010E2C6F38EC01F00F0E0301246FBD
:101A1C00256B266B276B286B296B2A6B2B6B2C6B1E
:101A2C0038EC01F0D00E0C6EC90E0D6E0D2EFED7DB
:101A3C000C2EFCD700000000D7EC03F08B80090EB5
:101A4C000B6E1E0E0C6EE40E0D6E0D2EFED70C2EB4
:0A1A5C00FCD70B2EFAD70000120091
:101A6600C69AFF0E0101776FFF0E786FFF0E796F32
:101A7600FF0E7A6F5E0E736F020E746F2D0E756F0A
:101A8600030E766F949A03010351040A02E19486C9
:101A960001D094969488C66AC79CC79E0351C61205
:101AA6000551C6120451C712055305E00651000A36
:101AB600D8B4C78C03D00653D8A4C78CC68A1200E4
:101AC6000101006B030E005D0CE2005103010425C9
:101AD600E16E000E0521E26E200EE66E0101002B7E
:101AE600F1D7005103010425E16E000E0521E26ED7
:101AF600E66A01010007005103010425066F000E86
:101B06000521076F0A0E046E03C300F055EC04F0BE
:101B160008C000F0300E002606C3E1FF07C3E2FF4F
:101B260000C0E6FF0A0E046E03C300F055EC04F095
:101B360000C003F30050000A01E103D001010007D1
:041B4600DAD71200D8
:101B4A0003C3F6FF04C3F7FF05C3F8FF0900F5CF87
:101B5A0001F00150000815E203C3F6FF04C3F7FFC2
:101B6A0005C3F8FF0900F5CF1AF306C31BF307C331
:101B7A001CF3E6EC06F0010E0327000E04230523EE
:041B8A00DFD712008F
:101B8E0003C304F004C305F004C002F005C003F063
:101B9E00044A052A05C300F006C301F00301054BF4
:101BAE00062B00C0E9FF01C0EAFF02C0E1FF03C03F
:101BBE00E2FFEECFE6FF02C0E9FF03C0EAFFEE52FE
:0E1BCE0001E0E2D703C300F004C301F01200EF
:101BDC0000C01AF001C019F0E1CF1BF0E2CF1CF0ED
:101BEC009DAA71D09EAA6FD0AECFFFF0ABA20FD042
:101BFC00AB98AECFFFF0AB88010E01016925006EEA
:101C0C00000E6A21016E00C069F101C06AF1ABA43B
:101C1C000FD00101AB9EAB8E010E6925006E000E3C
:101C2C006A21016E00C069F101C06AF1AECFFFF00C
:101C3C000001FF510D0A08E001018051000802E18A
:101C4C007F517E0801E31AD00101010E016F000ED5
:101C5C00026F9D9A810E7F25E16E020E8021E26E4D
:101C6C00E1CFE1FFE2CFE2FFE66A7FC101F380C181
:101C7C0002F37F6B806B0001FF6B25D0010180515B
:101C8C00000802E17F517E0804E2020E016F000E93
:101C9C00026F810E7F25E16E020E8021E26EE1CF94
:101CAC00E1FFE2CFE2FFFFC0E6FF7FC101F380C19D
:101CBC0002F3010E7F25006E000E8021016E00C024
:101CCC007FF101C080F1F2AA0CD0F2A40AD001017C
:101CDC002A0EAD6E010E6B27000E6C236D236E2346
:101CEC00F2941AC000F019C001F01BC0E1FF1CC037
:041CFC00E2FF1100F2
:101D000000C018F0156ED8CF16F0E0CF17F09DA0E8
:101D100019D09EA017D001016F4B702B0451705D3C
:101D200002E103516F5D09E39D906F6B706B010ED3
:101D3000716F000E726FCD909D900B0ECF6EDB0E0B
:101D4000CE6E9E901750E06E1650D86E153A15382C
:061D500018C000F01000B5
:101D5600ADEC18F09B6A700ED36E9B8CD26AD3B42E
:101D660001D0FDD7520E0B6E2B0E0C6E000E0D6EB3
:101D76000D2EFED70C2EFCD70B2EFAD70000FCEC4E
:101D860008F0520E0B6E2B0E0C6E000E0D6E0D2E05
:101D9600FED70C2EFCD70B2EFAD700008B80080E30
:101DA6000101036F000E046F899AB886030EB06EA8
:101DB600400EAF6EAC84D0EC08F0090E0B6E1E0E12
:101DC6000C6EE40E0D6E0D2EFED70C2EFCD70B2ED0
:101DD600FAD700000C0E03011A6F64EC04F0290E0A
:101DE6000B6E960E0C6E7F0E0D6E0D2EFED70C2E04
:101DF600FCD70B2EFAD7AF0E0001AD6F000EAE6FFB
:101E0600090E0101076F010E086F6EEC09F0D90E7D
:101E16000301036F300E046F000E056F50EC09F0DE
:101E26000101056B066B800E0619006E800E005CC4
:101E360002E10A0E055D20E2030E006E000E016E41
:101E460005C104F006C105F0E5EC05F0240E0024FA
:101E5600E96E000E0120EA6EE9CFE9FFEACFEAFF5C
:101E6600EECF03F3EECF04F3EECF05F350EC09F01B
:101E76000101054B062BD7D7A30E0B6E570E0C6E22
:101E8600020E0D6E0D2EFED70C2EFCD70B2EFAD79A
:101E960000006EEC09F0000E0001AB6FFA0EAC6F9D
:101EA600ADC003F3AEC004F30E0E0301056F300E92
:101EB600066F000E076F27EC09F0ABC003F3ACC04A
:101EC60004F3850E0301056F000E066F81EC08F022
:101ED600170E0001AD250301036F000E0001AE21B0
:101EE6000301046F850E056F000E066F050E076F62
:101EF600000E086F59EC08F0ADC003F3AEC004F352
:101F06003EEC08F09F90EB0E0301036F300E046F5A
:101F1600000E056F50EC09F030EC08F0670E030177
:101F2600036F2E0E046F000E056F50EC09F0010EC4
:101F36000301036F046B056B010E066F91DD1BDD5C
:101F4600690E036F300E046F000E056F50EC09F03A
:101F5600D7EC03F0520E0B6E2B0E0C6E000E0D6EB0
:101F66000D2EFED70C2EFCD70B2EFAD70000F28CC6
:101F7600D08EF28CF28E080E0101036F000E046FF4
:101F86006EEC09F0E30E0301036F2F0E046F000ED3
:101F9600056F50EC09F0D7EC03F0430E036F310EDA
:101FA600046F000E056F050E066F000E076FCADD83
:101FB6001D0E0301036F310E046F000E056F640ED4
:101FC600066F000E076FBEDD897AA30E0B6E570EE5
:101FD6000C6E020E0D6E0D2EFED70C2EFCD70B2EA0
:101FE600FAD70000897A1D0E0301036F2F0E046FC6
:101FF600000E056F50EC09F0D7EC03F0350E036FB9
:10200600310E046F000E056F050E066F000E076F8A
:1020160099DD07C103F308C104F34A0E0301056FF6
:10202600310E066F000E076F27EC09F007C11AF391
:1020360008C11BF362EC06F000C0A5F001C0A6F0D3
:1020460080C003F3850E046F000E056F39DD0001B5
:10205600A551010107250301036F0001A6510101E6
:1020660008210301046F850E056F000E066FB5EC9F
:1020760009F007C11AF308C11BF362EC06F000C0B1
:10208600A5F001C0A6F00050010107250301036F6A
:102096000150010108210301046F0A0E056F310E7C
:1020A600066F000E076F27EC09F00101006B79EC53
:1020B60009F000C0A5F001C0A6F03EEC06F0000E47
:1020C600046E000E056E480E066E840E076E6BECEF
:1020D60004F0000E046E000E056E000E066E890EEC
:1020E600076EFEEC04F000C081F001C082F002C071
:1020F60083F003C084F000C003F301C004F302C000
:1021060005F303C006F3850E0301076F000E086F83
:10211600010E096F3AEC0AF007C11AF308C11BF366
:1021260062EC06F000C0A5F001C0A6F00050010167
:1021360007250301036F0150010108210301046F04
:10214600850E056F000E066FB5EC09F007C11AF390
:1021560008C11BF362EC06F000C0A5F001C0A6F0B2
:102166000050010107250301036F015001010821F9
:102176000301046F520E056F310E066F000E076FD6
:1021860027EC09F007C103F308C104F33EEC08F09D
:102196006EEC09F007C11AF308C11BF362EC06F0F6
:1021A60000C0A5F001C0A6F0897A0101056B066B97
:1021B600800E0619006E800E0001A619005C03E170
:1021C600A5510101055D1DE2010105510725E96ED5
:1021D60006510821EA6EE9CFE9FFEACFEAFFEE50A1
:1021E600B00A0CE105510725E16E06510821E26EA1
:1021F600E1CFE1FFE2CFE2FF7E0EE66E054B062B56
:10220600D7D70101090E076F010E086F07C103F347
:1022160008C104F3960E0301056F000E066F24EC49
:102226000AF0A30E0B6E570E0C6E020E0D6E0D2EDF
:10223600FED70C2EFCD70B2EFAD70000D7EC03F0F6
:102246003C0E036F310E046F000E056F050E066F10
:10225600000E076F77DCAF0E0001AD6F000EAE6F9C
:10226600ADC003F3AEC004F33FC005F340C006F3B0
:1022760041C007F327EC09F0FC0E0301036F300E93
:10228600046F000E056F50EC09F0ADC003F3AEC04D
:1022960004F33EEC08F06EEC09F0ADC01AF3AEC0E4
:1022A6001BF362EC06F000C0A5F001C0A6F0010128
:1022B600056B066B800E0619006E800E0001A619CE
:1022C600005C03E1A5510101055D25E2010105510F
:1022D6000001AD25E96E010106510001AE21EA6E4D
:1022E600E9CFE9FFEACFEAFFEE50B00A10E10101BB
:1022F60005510001AD25E16E010106510001AE2137
:10230600E26EE1CFE1FFE2CFE2FF7E0EE66E010173
:10231600054B062BCFD7AF0E0001AD6F000EAE6F8B
:10232600ADC003F3AEC004F3960E0301056F000EB5
:10233600066F24EC0AF0A30E0B6E570E0C6E020EFF
:102346000D6E0D2EFED70C2EFCD70B2EFAD70000E5
:102356000001A99B806B500E226E000E236E26ECA8
:102366000CF0D7EC03F02E0E036F310E046F000E47
:10237600056F020E066F000E076FA5EC0DF000014B
:10238600A9AB04D107C103F308C104F34E0E030140
:10239600056F310E066F000E076F27EC09F007C1B7
:1023A6001AF308C11BF362EC06F000C0A5F001C0E9
:1023B600A6F080C003F3850E046F000E056F63EC74
:1023C6000DF00001A551010107250301036F00016E
:1023D600A651010108210301046F850E056F000E49
:1023E600066FB5EC09F007C103F308C104F33EEC30
:1023F60008F0090E03011A6F64EC04F0090E0101DE
:10240600076F010E086F07C103F308C104F3260E18
:102416000301056F310E066F000E076F27EC09F0FA
:102426000101006B79EC09F000C0A5F001C0A6F02F
:102436003EEC06F0000E046E000E056E480E066EAB
:10244600840E076E6BEC04F0000E046E000E056E33
:10245600000E066E890E076EFEEC04F000C081F0D9
:1024660001C082F002C083F003C084F000C003F311
:1024760001C004F302C005F303C006F3850E030191
:10248600076F000E086F010E096F3AEC0AF007C1DC
:102496001AF308C11BF362EC06F000C0A5F001C0F8
:1024A600A6F00050010107250301036F0150010149
:1024B60008210301046F850E056F000E066FB5EC4B
:1024C60009F007C11AF308C11BF362EC06F000C05D
:1024D600A5F001C0A6F00050010107250301036F16
:1024E6000150010108210301046F560E056F310EDC
:1024F600066F000E076F27EC09F007C103F308C14A
:1025060004F33EEC08F06EEC09F007C11AF308C1BB
:102516001BF362EC06F000C0A5F001C0A6F00101B5
:10252600056B066B800E0619006E800E0001A6195B
:10253600005C03E1A5510101055D1DE201010551A4
:102546000725E96E06510821EA6EE9CFE9FFEACFD1
:10255600EAFFEE50B00A0CE105510725E16E06517F
:102566000821E26EE1CFE1FFE2CFE2FF7E0EE66EEA
:10257600054B062BD7D707C103F308C104F322C0C6
:1025860005F323C006F324EC0AF04FD0AF0E00018A
:10259600AD6F000EAE6FADC003F3AEC004F33EECFC
:1025A60008F06EEC09F00101056B066BADC01AF37D
:1025B600AEC01BF362EC06F0800E01010619026E36
:1025C600800E0118025C02E10050055D24E205510F
:1025D6000001AD25E96E010106510001AE21EA6E4A
:1025E600E9CFE9FFEACFEAFFEE50B00A10E10101B8
:1025F60005510001AD25E16E010106510001AE2134
:10260600E26EE1CFE1FFE2CFE2FF7E0EE66E010170
:10261600054B062BCBD7ADC003F3AEC004F322C0E7
:1026260005F323C006F324EC0AF0520E0B6E2B0EB4
:102636000C6E000E0D6E0D2EFED70C2EFCD70B2E3B
:10264600FAD700000001802BA30E0B6E570E0C6EFE
:10265600020E0D6E0D2EFED70C2EFCD70B2EFAD7C2
:102666000000000E0101021902E1010E0119D8A4B1
:102676005BD1810E0301036F020E046F1D0E056F01
:10268600000E066FE5EC09F000C0A7F001C0A8F047
:10269600000E026E0150025C02E1005000083FE2AB
:1026A600810E03011A6F020E1B6F62EC06F0800E9C
:1026B600026E800E0118025C02E1005006082FE24D
:1026C600810E1A6F020E1B6F62EC06F000C0A5F0B9
:1026D60001C0A6F0800E026E800E0118025C02E1B7
:1026E600005006081CE2800E0001A619006E800E3E
:1026F600005C02E1540EA55D12E25B0E0301036F5E
:10270600000E046F3EEC08F0ADC003F3AEC004F358
:10271600850E0301056F020E066FC7EC0DF003016F
:10272600810E036F020E046F770E056F000E066FA3
:10273600E5EC09F000C0A7F001C0A8F0000E026E9B
:102746000150025C02E10050000815E20001A98B6D
:10275600810E03011A6F020E1B6F62EC06F000C0B9
:10276600A5F001C0A6F0990E036F300E046F000E9F
:10277600056F50EC09F0810E0301036F020E046F22
:102786004B0E056F000E066FE5EC09F000C0A7F0D2
:1027960001C0A8F0000E026E0150025C02E100507A
:1027A60000080BE20001A99B860E0301036F2F0EA2
:1027B600046F000E056F50EC09F0810E0301036FE4
:1027C600020E046F540E056F000E066FE5EC09F05D
:1027D60000C0A7F001C0A8F0000E026E0150025C16
:1027E60002E100500008D8B09DD0810E03011A6F97
:1027F600020E1B6F62EC06F000C0A5F001C0A6F049
:10280600800E026E800E0118025C02E1005006087E
:10281600D8B088D001017B6B7C6B056B066B060E0E
:102826000001A55D016E000EA659026E800E010123
:102836000619006E800E0218005C02E10150055D6B
:1028460023E2870E0525E96E020E0621EA6EE9CF20
:10285600E9FFEACFEAFFEECF01F0300E015C11E3AB
:10286600870E0525E96E020E0621EA6EE9CFE9FF1D
:10287600EACFEAFFEECF01F00150390802E37B4BC5
:102886007C2B054B062BCBD7060E0001A55D016EF2
:10289600000EA659026E01017C51021802E1015098
:1028A6007B1940E1870E0301036F020E046F53ECA0
:1028B6000CF000C07DF101C07EF1800E026E800E2C
:1028C6000118025C02E1005001080FE2800E0101CE
:1028D6007E19006E800E020A005C02E1000E7D5D2C
:1028E60004E27DC122F07EC123F0C50E0301036F11
:1028F600300E046F000E056F50EC09F022C003F392
:1029060023C004F3850E0301056F000E066F81ECEC
:1029160008F0850E0301036F000E046F3EEC08F00D
:0C2926006EEC09F026EC0CF01CD5FFD77D
:10315A0010EE1DF0630E006E010E016E320EF66E59
:0E316A002D0EF76E000EF86E1FEC09F012002D
:102932000000000000000000000000000000000095
:102942000000000000000000000000000000000085
:102952000000000000000000000000000000000075
:102962000000000000000000000000000000000065
:102972000000000000000000000000000000000055
:102982000000000000000000000000000000000045
:102992000000000000000000000000000000000035
:1029A2000000000000000000000000000000000025
:1029B2000000000000000000424242000042424289
:1029C200844221000084422100E700000000E70069
:1029D2002142840000214284010204081020408028
:1029E2008040201008040201AA55AA55AA55AA55EA
:1029F200815A244242245A810058640404645800D3
:102A02000C1222444422120C7E81A59191A5817E52
:102A12007E8195A1A195817E20342AE1E12A34208C
:102A220010F884828284F810985CB65F5FB65C9876
:102A320000000000000000000000009F00000000F5
:102A4200000007000007000000247E24247E2400EA
:102A520000242A7F2A1200000043231008C4C20067
:102A6200007689956260800000000905030000007D
:102A72000000182442810000000081422418000056
:102A82000014087F081400000010107C10100000D1
:102A920000001090700000000010101010101000C4
:102AA2000000C0C000000000004020100804020026
:102AB200007EA19189857E0000848281FF80800052
:102AC2000082C1A1918986000042818989897600AC
:102AD2000030282422FF2000008F89898989710013
:102AE200007E9191919160000001E11109050300BE
:102AF20000768989898976000006898989493E009C
:102B02000000006666000000000000AC6C000000DF
:102B1200000008142241000000242424242424005C
:102B22000000412214080000000201B10906000061
:102B3200000000000000000000FE21212121FE0013
:102B420000FF898989897600007E81818181420026
:102B520000FF818181423C0000FF898989818100D7
:102B620000FF090909010100007E81819191F200B3
:102B720000FF08080808FF00008181FF8181000032
:102B820000408081817F010000FF181824428100EB
:102B920000FF80808080800000FF02040402FF00AA
:102BA20000FF04081020FF00007E818181817E00E9
:102BB20000FF090909090600007E8181A141BE00CA
:102BC20000FF0919294986000086898989897100CF
:102BD200000101FF01010000007F808080807F00F2
:102BE200003F408080403F00007F806060807F0027
:102BF20000C324181824C300000708F0F0080700D7
:102C020000C1A1918985830000FF8181000000003D
:102C1200001516FC161500000000008181FF00005F
:102C22000004020102040000008080808080800095
:102C320000010204000000000020545454780000F7
:102C4200007E4848483000000038444444200000D8
:102C520000304848487E0000003C4A4A4A0C0000C6
:102C620000107C1202040000000C5252523E00007E
:102C7200007E100808700000000000447D40000043
:102C820000204040443D00000000FE20508800002B
:102C9200000082FE808000000078041804780000A2
:102CA200007C0804047800000038444444380000E2
:102CB200007C14140800000000081414187C0000A2
:102CC200007C08040408000000485454240000005A
:102CD20000043E4440200000003C4040207C0000B4
:102CE200001C2040201C0000003C4030403C000002
:102CF200004428102844000000000C50503C000002
:102D0200004464544C4400000000083641000000B6
:102D1200000000FF00000000000000413608000033
:102D220000000609090600000010385410101000B7
:052D32004D73673D0038
:022D3700640036
:102D3900503000E22D00A82E00952D00E52E00B0A0
:102D49003000262E00532F00B62F0081300081302D
:072D590000333000143100CB
:092D600054454D505F4F464600FA
:072D690053706565643D0035
:102D70000D0A2068656C6C6F2C20692067657420D3
:0C2D8000796F7572204D7367210D0A00F9
:082D8C0054454D505F4F4E000D
:012D94000F2F
:102D950020536F75726365203A205F3138463436AB
:102DA5004B32325F746573745F4F6C645F4D61784D
:102DB50037313231395F38784D61747269636538FE
:102DC50078385F535049315F486172647761726545
:0D2DD5005F3139303632342E63200D0A0094
:102DE200204469726563746F7279203A20433A5CB9
:102DF2005F4D696B726F435C5F4D657350726F6AB2
:102E02006574735F4D696B726F435C5F4D617837B8
:102E12003231395F385F6D61747269636538783851
:042E2200200A0D0075
:102E26002038204D617472696365203878382072C5
:102E36006163636F7264656D656E74207665727426
:102E46006963616C2048415554207665727320424F
:102E5600617320737572204D4158373132390A0D2E
:012E6600006B
:102E6700496E69742053504920416476616E6365E9
:102E77006420484152445741524520205243332051
:102E87002853434B292C20524335202853444F2C99
:102E970029206574205243302028435329200D0AE6
:012EA700002A
:102EA8002050726F6A6574203A2031384634364BA8
:102EB80032325F4D4158373231395F6F6C645F3859
:102EC800785F4D61745F3878385F535049315F4897
:0D2ED800617264772E6D63707069720A007C
:102EE50020436F6E666967204269747320503138DC
:102EF5004634364B32325F466F73635F696E746575
:102F0500726E655F313678345F36344D487A2E639C
:082F150066677363680A0D0092
:102F1D0020446973706C6179203C4A3D202020303B
:102F2D00202054B0414D423D2034382E3320B04343
:102F3D003E20737572206D61747269636573204CE8
:062F4D006564730D0A002B
:102F53002053616973697220756E206E6F75766593
:102F63006175204D73672061766563206C652074FD
:102F730065726D696E616C20766961204D73673D82
:032F83000D0A0034
:102F86000D0A204F4B2C2054656D706572206973B5
:102F9600204F4646210D0A5265746F757220617581
:102FA60020646973706C617920747874200D0A004E
:102FB600204D6F64652054656D706572617475721D
:102FC6006520617665632054454D505F4F4E206FF6
:0D2FD600752054454D505F4F46460D0A00D2
:102FE30020446973706C6179203C3031323334355D
:102FF30036373E207375722038206D6174726963B1
:0B3003006573204C656473200D0A000B
:10300E000D0A20436C6F636B20696E697469616C85
:10301E006520696E20203D20202E2E2E20204B680C
:05302E007A200D0A00EC
:10303300B02AB0204C45204A4F5552204C452050D1
:0D3043004C5553204C4F4E4720B02AB00092
:10305000204D696B726F6320372E31302031384636
:0930600034364B3232200A0D0017
:1030690020436C656172204D617472696365203813
:0830790078203878380D0A00B8
:103081002043414E4943554C4520454E204A554920
:083091004E20323031392000DD
:103099000D0A204F4B2C2054656D706572206973A1
:0730A900204F4E210D0A002B
:1030B00020506F77657220537570706C7920332EB5
:0530C00036560A0D0068
:1030C5000D0A204368616E6765205370656564204D
:0430D500546F200014
:1030D9002050726573656E746174696F6E203A0D64
:0230E9000A00DB
:1030EB0020496E69742041444320454130200D0A2C
:0130FB0000D4
:0E30FC00204D6573736167652039203A20000E
:0A310A00202054B0414D423D20004A
:09311400207878787878782000A2
:09311D003031323334353637000D
:0831260054B02E416D623D0022
:07312E0020202020202000DA
:0731350020202020202000D3
:07313C0020202020202000CC
:0731430020202020202000C5
:04314A004A3D2000DA
:04314E004A3D2000D6
:0431520020B0430066
:03315600B0430083
:020000040030CA
:0D000100381E3CFF9880FF0FC00FE00F403D
:0200000400F00A
:100000007061756C666A756A696F40667265652EA7
:100010002E667220200D0A002020202020202000A3
:1000200031382F31322F32303136200D0A00200086
:10003000FFFFFFFFFFFFFFFFFFFFFFFFFFFFFFFFD0
:10004000FFFFFFFFFFFFFFFFFFFFFFFFFFFFFFFFC0
:10005000FFFFFFFFFFFFFFFFFFFFFFFFFFFFFFFFB0
:10006000FFFFFFFFFFFFFFFFFFFFFFFFFFFFFFFFA0
:00000001FF
